:020000040800F2
:1000000000500020CD0B0008450A0008490A0008EE
:100010004D0A0008510A0008550A000800000000B7
:10002000000000000000000000000000590A000865
:100030005D0A000800000000610A0008650A000867
:10004000110C0008110C0008110C0008110C00081C
:10005000110C0008110C0008110C0008110C00080C
:10006000110C0008110C0008110C0008110C0008FC
:10007000110C0008110C0008110C0008110C0008EC
:10008000110C0008110C0008110C0008110C0008DC
:10009000110C0008110C0008110C0008110C0008CC
:1000A000110C0008110C0008110C0008110C0008BC
:1000B000110C0008110C0008110C0008110C0008AC
:1000C000110C0008110C0008110C0008110C00089C
:1000D000110C0008110C0008110C0008110C00088C
:1000E000110C0008110C0008110C000800000000A1
:1000F0000000000000000000000000000000000000
:0C01000000000000000000005FF808F1A3
:10010C0040F21403C2F200031A780AB901201870E5
:10011C00704700BF40F21400C2F2000008B503683B
:10012C002BB140F20003C0F2000303B1984708BDA5
:10013C00CB7810B413F0100F18BF8A7803F00F0CA3
:10014C0018BF4CEA020C0A8812F0FF0F29D002F0FB
:10015C0001040168002C40F0258102F00204002CFF
:10016C0040F0FD8002F00404002C40F0098102F004
:10017C000804002C40F0AE8002F01004002C40F07B
:10018C00BA8002F02004002C40F0C68002F040043B
:10019C00002C40F0D28002F08004002C40F014813E
:1001AC000160FF2A20D902F480744168002C27D109
:1001BC0002F40074002C32D102F48064002C3DD186
:1001CC0002F40064002C48D102F48054002C53D16A
:1001DC0002F40054002C5ED102F48044002C69D14E
:1001EC0002F4004212B9416010BC7047282B6CF32A
:1001FC001F7108BF4261F6D0482B08BF0261F2E7BD
:10020C0021F00F01282B4CEA010108BF4461CFD02B
:10021C00482B08BF046102F40074002CCCD021F0F0
:10022C00F001282B41EA0C1108BF4461C4D0482BC3
:10023C0008BF046102F48064002CC1D021F4706109
:10024C00282B41EA0C2108BF4461B9D0482B08BFC8
:10025C00046102F40064002CB6D021F47041282B08
:10026C0041EA0C3108BF4461AED0482B08BF046191
:10027C0002F48054002CABD021F47021282B41EADD
:10028C000C4108BF4461A3D0482B08BF046102F4A1
:10029C000054002CA0D021F47001282B41EA0C5101
:1002AC0008BF446198D0482B08BF046102F4804415
:1002BC00002C95D021F07061282B41EA0C6108BF0D
:1002CC0044618DD0482B02F4004208BF0461002A1F
:1002DC0089D08BE721F47041282B41EA0C3108BFFF
:1002EC0044613FF449AF482B08BF046102F010048D
:1002FC00002C3FF446AF21F47021282B41EA0C412D
:10030C0008BF44613FF43DAF482B08BF046102F0C5
:10031C002004002C3FF43AAF21F47001282B41EA61
:10032C000C5108BF44613FF431AF482B08BF046146
:10033C0002F04004002C3FF42EAF21F07061282B0A
:10034C0041EA0C6108BF44613FF425AF482B08BF5C
:10035C00046102F08004002C3FF422AF34E021F061
:10036C00F001282B41EA0C1108BF44613FF4FAAEAE
:10037C00482B08BF046102F00404002C3FF4F7AED4
:10038C0021F47061282B41EA0C2108BF44613FF431
:10039C00EEAE482B08BF046102F00804002C3FF4B9
:1003AC00EBAE97E721F00F01282B4CEA010108BFB7
:1003BC0044613FF4D2AE482B08BF046102F0020442
:1003CC00002C3FF4CFAECAE7282B6CF31F7108BF8B
:1003DC0044613FF4E5AE482B08BF0461E0E600BF82
:1003EC00042202214FF0FF33C270817003807047EA
:1003FC00836819420CBF002001207047806880B2CE
:10040C00704700BFC36819420CBF00200120704721
:10041C00C06880B2704700BF01617047416170478E
:10042C000AB9416170470161704700BFC1607047F4
:10043C0041F480338361816183618369836970478F
:10044C0040F20002C4F2010210B44FF6807314683B
:10045C00C0F2000304EA030C41EA001141EA0C0368
:10046C00136010BC704700BF40F21C03C4F2202381
:10047C001860704740F200030028C4F20103B4BFB7
:10048C00DA695A6800F44013B3F5401F10B41FFA30
:10049C0080FC25D010F4801F19D0C0F30343032433
:1004AC0014FA03F322EA030242F0706229B1430DFD
:1004BC0019010CFA01FC42EA0C02002840F200007F
:1004CC00C4F20100B4BFC261426010BC7047430D5E
:1004DC001B010CFA03F322EA030242F07062E5E717
:1004EC0040F20003C4F201035C6822F0706224F055
:1004FC0070645C60DAE700BF01F0030310B40F22F4
:10050C009C00A24010FA04F3890840F20004C4F2E3
:10051C000104023154F8210020EA020244F821209F
:10052C0054F82120134344F8213010BC704700BF0D
:10053C0040F2DC03C4F2202318607047012001460E
:10054C0010B500F00BFA01200021BDE8104000F0BE
:10055C0005BA00BF40F60003C4F20103984210B57F
:10056C0030D040F60041C4F20101884234D041F24F
:10057C000002C4F20102904238D041F2004CC4F2A5
:10058C00010C60453CD041F60003C4F201039842D3
:10059C0040D041F60041C4F20101884244D042F2FD
:1005AC000002C4F20102904200D010BD01214FF4B0
:1005BC00807000F0D3F94FF480700021BDE810403A
:1005CC0000F0CCB90420012100F0C8F9042000216E
:1005DC00BDE8104000F0C2B90820012100F0BEF9BE
:1005EC0008200021BDE8104000F0B8B9102001210E
:1005FC0000F0B4F910200021BDE8104000F0AEB9B5
:10060C002020012100F0AAF920200021BDE8104093
:10061C0000F0A4B94020012100F0A0F940200021F5
:10062C00BDE8104000F09AB98020012100F096F945
:10063C0080200021BDE8104000F090B941F2000389
:10064C00C4F20203186840F2000C40F001021A6078
:10065C005968CFF6FF0C01EA0C0058601A6822F0BA
:10066C00847C2CF480311960186820F480221A6084
:10067C0059684FF41F0221F4FE0058609A607047CD
:10068C0041F20003C4F202031968B0F5803F21F473
:10069C0080321A60196821F480221A6007D0B0F5F4
:1006AC00802F03D1186840F4A021196070471A6894
:1006BC0042F480301860704782B041F20001002390
:1006CC000193C4F202010A680198431C019301983A
:1006DC00B0F5A06F02D012F4003FF4D041F200024A
:1006EC00C4F202021168C1F3404002B0704700BF6F
:1006FC0041F20003C4F202031A6822F0F80141EA45
:10070C00C0021A60704700BF40F20003C4F24223DB
:10071C001860704741F20003C4F202035A6822F4D5
:10072C007C1C40EA0C020A435A60704740F260039A
:10073C00C4F242231860704741F20003C4F2020372
:10074C005A6822F0030140EA01025A60704700BF68
:10075C0041F20003C4F20203586800F00C00704729
:10076C0041F20003C4F202035A6822F0F00140EA9D
:10077C0001025A60704700BF41F20003C4F2020349
:10078C005A6822F4E06140EA01025A60704700BFE7
:10079C0041F20003C4F202035A6822F4605141EAA8
:1007AC00C0025A60704700BF49B941F20901C4F256
:1007BC00020191F800C02CEA00000870704741F269
:1007CC000903C4F202031A7810431870704700BF73
:1007DC0040F2D803C4F242231860704741F2000380
:1007EC00C4F202035A6822F4404140EA01025A6002
:1007FC00704700BF41F220030022C4F2020301281B
:10080C001A701A7004D0042801D105201870704792
:10081C001870704740F28043C4F24223186070474E
:10082C0041F20003C4F20203196A40EA01021A629F
:10083C00704700BF40F23C43C4F24223186070473B
:10084C0041F20003C4F202035A6810B402F00C0225
:10085C00042A01D0082A2ED041F20021C0F27A01DC
:10086C00016041F20002C4F20202546840F200033B
:10087C00C2F20003C4F3031C13F80CC021FA0CF1F0
:10088C0041605468C4F3022C13F80C4031FA04F4A0
:10089C0084605468C4F3C22C13F80CC021FA0CF118
:1008AC00C1605268C2F38132D3181A7CB1FBF2F1E9
:1008BC00016110BC70475A685C68C2F38341023115
:1008CC0014F4803F0BD05B6813F4003F07D141F266
:1008DC000024C0F27A0404FB01F10160C1E740F688
:1008EC00001CC0F23D0C0CFB01F10160B9E700BF2C
:1008FC0041B941F20001C4F202014B6923EA000044
:10090C004861704741F20003C4F202035A69104374
:10091C005861704741B941F20001C4F202018B6980
:10092C0023EA00008861704741F20003C4F202031D
:10093C009A6910439861704741B941F20001C4F2C1
:10094C000201CB6923EA0000C861704741F2000341
:10095C00C4F20203DA691043D861704741B941F21D
:10096C000001C4F20201CB6823EA0000C8607047A2
:10097C0041F20003C4F20203DA681043D8607047F6
:10098C0041B941F20001C4F202010B6923EA0000F3
:10099C000861704741F20003C4F202031A69104364
:1009AC001861704740F24043C4F24223186070470C
:1009BC0040F24C03C4F242231860704741F2070323
:1009CC00C4F20203187070474309012B0ED0022B9E
:1009DC0041F20003C4F202030CBF1B6A5B6A00F015
:1009EC001F0133FA01F000F00100704741F20003DF
:1009FC00C4F202031B6800F01F0133FA01F000F08F
:100A0C000100704741F20003C4F20203586A40F03F
:100A1C0080725A62704700BF41F20001C4F20201B9
:100A2C008B6818420CBF00200120704741F20A036A
:100A3C00C4F2020318707047704700BFFEE700BF96
:100A4C00FEE700BFFEE700BFFEE700BF704700BF38
:100A5C00704700BF704700BF704700BF82B0019065
:100A6C00019B2BB1019A511E019101980028F9D1DB
:100A7C0002B0704710B5FFF7E1FD4FF48030FFF77F
:100A8C00FFFDFFF719FE40F21803C2F20003012824
:100A9C000446187000D010BD0020FFF761FE002046
:100AAC00FFF776FE4FF48060FFF766FE4FF4803060
:100ABC000021FFF72FFE2046FFF738FE3920FFF705
:100ACC0083FF0028FAD00220FFF736FEFFF740FE26
:100ADC000828FBD110BD00BF08B541F20000C4F2DC
:100AEC0001002021FFF798FC41F20000C4F2010044
:100AFC001021FFF793FC40F60040C4F20100802166
:100B0C00FFF78AFC40F60040C4F201004FF48071FC
:100B1C00FFF784FC4FF6FE73C0F2FF03023BFDD1DE
:100B2C0041F20000C4F201001021FFF775FC41F204
:100B3C000000C4F201002021FFF770FC40F60040D9
:100B4C00C4F201004FF48071FFF766FC40F60040E0
:100B5C00C4F201008021FFF761FC4FF6FE73C0F276
:100B6C00FF03023BB9D0FCE770B5FFF783FF102001
:100B7C000121FFF7CFFE40F21C0408200121FFF7F2
:100B8C00C9FEC2F2000441F20000012610252146E4
:100B9C004FF03002C4F201002280A670E570FFF71E
:100BAC00C7FA40F600404FF4C073C4F2010021466E
:100BBC00A670E5702380BDE87040FFF7B9BA00BF9E
:100BCC00002103E00A4B5B584350043109480A4B9F
:100BDC0042189A42F6D3094A02E0002342F8043B39
:100BEC00074B9A42F9D3FFF7BFFFFFF775FF70472A
:100BFC00340C000800000020140000201400002019
:100C0C0020000020FEE70000F8B500BFF8BC08BCCF
:100C1C009E467047F8B500BFF8BC08BC9E467047AE
:040C2C00210100089A
:040C30000D010008AA
:100C3400000000000102030401020304060708097E
:040C44000204060898
:0400000508000BCD17
:00000001FF
